:020000040000FA
:0400000000EF7CF0A1
:04F7FC000000000009
:10F80000ADEF7FF000C0E5FF01C0E5FF00EE62F064
:10F8100002EC7FF0006E00C0F3F000C0F4F002ECE8
:10F820007FF0006E0001E96F00500001F42702EC48
:10F830007FF0006E0001E86F00500001F42702EC39
:10F840007FF0006E00C0F5F000500001F4270001C9
:10F85000F551040A24E10001E951D8A4DBD0E851B4
:10F86000D8A4D8D00001F351020A01E0D3D002ECB1
:10F870007FF0006E0001EB6F00500001F42702ECF6
:10F880007FF0006E0001EA6F00500001F42702ECE7
:10F890007FF0006E0001F427F451D8A4B3D000012A
:10F8A000F551010A20E102EC7FF0006E0001F4271F
:10F8B000F451D8A4A7D00001F2B3B9EC7DF098ECD4
:10F8C0007FF00001F2A50BD0C00E0001E46FF70E2F
:10F8D000E56FE66BE76BB9EC7DF098EC7FF0590EC5
:10F8E00070EC7FF09AD00001EB510001E71914E1B0
:10F8F0000001EA510001E6190FE10001E9510001A0
:10F90000E5190AE1C00E0001E815006EC00E000105
:10F91000E415016E00180FE00001F2A302D0B9EC6B
:10F920007DF098EC7FF0E8C0E4F0E9C0E5F0EAC0D3
:10F93000E6F0EBC0E7F00001F551040A01E15ED00A
:10F940000001F551D8A462D00001F351D8B456D0CB
:10F950000001EB51D8A45AD0EA51E00BD8A456D0FC
:10F960000001F2A912D00001F3514EEC7EF0400EDE
:10F97000A3EC7FF00001E9514EEC7EF00001E8516C
:10F980004EEC7EF0200EA3EC7FF0EAC0F8FFE9C059
:10F99000F7FFE8C0F6FF000100EE6AF028EE00F085
:10F9A000E8513F0BD926D8B0DA2ADD5202EC7FF0BD
:10F9B0000001F427DC6E0900F55C05E00001F2832C
:10F9C0002A0EA3EC7FF00001F2A906D0DF504EEC26
:10F9D0007EF0200EA3EC7FF00001F32FE7D702ECBE
:10F9E0007FF0006E0001F427F45108E00001E469A3
:10F9F000E569E669E7690001F29304D0580E70ECFE
:10FA00007FF00BD07A0E70EC7FF007D0750E70ECA3
:10FA10007FF003D06C0E70EC7FF0E4CF01F0E4CF08
:10FA200000F01200FF0E926E936E946E966ED8ECFC
:10FA30007FF0970ED56E8B809490B06A3F0EAF6EBC
:10FA4000B886AC8AAC84AC8CAC90AB8CAB8E00012D
:10FA5000E46BE56BE66BE76B0001E86BE96BEA6B67
:10FA6000EB6B98EC7FF00001F26B93988A888B9097
:10FA7000AB984B0EA3EC7FF0B7EC7FF00001EC6B82
:10FA8000ED6B8BB002D0B7EC7FF00001606BC2EC85
:10FA90007EF000016051D8B45CD08B90AB988AA8FE
:10FAA00002D08A9801D08A8861C000F00050520AC2
:10FAB00003E161EC7FF00BD00050500A03E152ECFF
:10FAC0007FF005D00050560A02E17EEC7EF0000186
:10FAD000F2A13FD00050450A03E140EC7FF039D05D
:10FAE00000503A0A03E102EC7CF033D00050720A75
:10FAF00003E1A1EC7EF02DD00050410A03E1DBECE4
:10FB00007FF027D00050760A24E1006A000162519C
:10FB1000300A01E1002A0050D880E866D890006AD7
:10FB200000360050010BE838E840F46E0001F25155
:10FB3000F70BF410F26F320E0001625D006A0036BE
:10FB40000050010BE838F46E0001F251EF0BF41095
:10FB5000F26F0001F2B195D70001ED51800F800FD7
:10FB600002E1A10EEC5DD8A08CD7DBEC7FF089D749
:10FB7000120000C0E5FF01C0E5FF02C0E5FF03C0C1
:10FB8000E5FF0001E4513F0B04E0210EA3EC7FF000
:10FB90007CD00001E75103E1E651E00BD8A475D019
:10FBA000E4C000F0E5C001F0026A036A0350800F70
:10FBB000800F08E1000E025C05E1F80E015C02E135
:10FBC000000E005C01E361D0E4C000F0E5C001F08C
:10FBD000E6C002F0E7C003F000500110021003106D
:10FBE00013E100C8E0F001C8E1F002C8E2F003C888
:10FBF000E3F00801006BEF0E016F7C0E026FF00E58
:10FC0000036F0001F28515D00050C00A07E10150D2
:10FC1000F70A04E1025002E1035001E00AD0E0C01B
:10FC20003CF8E1C03DF8E2C03EF8E3C03FF8000117
:10FC3000F2950001F2A70BD0200EA3EC7FF000019B
:10FC4000E5514EEC7EF00001E4514EEC7EF0E6C052
:10FC5000F8FFE5C0F7FFE4C0F6FF940EBFEC7FF0BD
:10FC60000A0008EE00F00001080EEE6F080EEF6FBC
:10FC7000EE50F56E0F00EF2FFBD7840E80D9EE2FDC
:10FC8000F5D7A694570E70EC7FF0E4CF03F0E4CFE5
:10FC900002F0E4CF01F0E4CF00F0120000C0E5FF75
:10FCA00001C0E5FF02C0E5FF006E00380F0B026ED9
:10FCB000300E0224016E3A0E015C05E30150026E23
:10FCC000070E0224016E0150A3EC7FF00F0E00140A
:10FCD000006E300E0024016E3A0E015C05E3015007
:10FCE000006E070E0024016E0150A3EC7FF0E4CFFC
:10FCF00002F0E4CF01F0E4CF00F0120000EE62F079
:10FD0000000160050001EF6FEF07010EEE6FEE518D
:10FD1000D2EC7FF004E10A0EEE6FD2EC7FF0EE5CE5
:10FD2000D8A41200EE2BEF2FF2D7EE51D2EC7FF0D9
:10FD3000D8A41200560E70EC7FF00001F281F2950B
:10FD4000120000C0E5FF00EE62F002EC7FF0F76EFB
:10FD500002EC7FF0F66E720EA3EC7FF0200EA3ECA7
:10FD60007FF0100E006E0900F5504EEC7EF0200E74
:10FD7000A3EC7FF0002EF7D70A0EA3EC7FF0E4CFC0
:10FD800000F01200CCEC7FF0000100EE60F0E2EC3D
:10FD90007EF0E86614D0AE50EE6EEE6FEF6FD8B422
:10FDA0000ED0CCEC7FF0E2EC7EF0E86608D0AE50EE
:10FDB000EE6EEF27EE2FF5D7EF53D8B41200000107
:10FDC000606B12009EBA08D0F2A4FCD70001EC3F91
:10FDD00001D0ED2BE86815D08A98ABB202D0ABA465
:10FDE00004D0B7EC7FF0E8680CD0ABA009D0AE50DF
:10FDF00005E1CCEC7FF0E2EC7EF003D0DBEC7FF0B1
:10FE0000E86A12000001EECFEEF0EECFEFF0D00E78
:10FE1000EE27EF27F60EEE25F90ED8B0EE27F60EF8
:10FE2000EF25F90ED8B0EF27EE39EF25E850120094
:10FE300000EE68F000016051F80F0001EE6F09E07C
:10FE4000F05D07E3EE50A86E8CEC7FF0A92AEE2F50
:10FE5000F9D7A86A8CEC7FF0120000C0E5FF01C062
:10FE6000E5FF006A00EE62F0060E016EEE5000261D
:10FE7000012EFCD70050E4CF01F0E4CF00F01200D7
:10FE800000EE61F0000160510001EE6F07E0EE0747
:10FE900005E0EE50A3EC7FF0EE2FFBD70A0EA3ECAB
:10FEA0007FF012002DEC7FF0B80A0AE1010EA96E76
:10FEB000080E0001F06F18EC7FF0500E70EC7FF030
:10FEC00012002DEC7FF0A00A0AE10A0EA96E100EB6
:10FED0000001F06F18EC7FF0520E70EC7FF0120012
:10FEE00000C0E5FF006E200EA3EC7FF00050A3ECF5
:10FEF0007FF00A0EA3EC7FF0E4CF00F01200700E4A
:10FF0000D36E9B8C0F013A9FFF0E926893689468A2
:10FF10009668626AF19E1200A69EA69CA684550E63
:10FF2000A76EAA0EA76EA682A6B2FED7A69412004E
:10FF30000001F2930001400EEE6F08EE00F0EE6853
:10FF4000EE2FFDD7120000C0E5FF006E9EA8FED781
:10FF500000C0ADFFE4CF00F0120017EEFFF027EE77
:10FF6000FFF0F86AA68EA69C12EC7DF0FFD7ACA23B
:10FF7000FED78B80AE50AE50AB98AB881200A66E09
:10FF8000550EA76EAA0EA76EA6821200C8EF7FF0CC
:10FF900012EC7DF0CAEF7FF0F70ED76EF80ED66E3A
:10FFA000F2941200A96EA69CA69EA680A8501200EC
:0AFFB0007FEC7FF01200FEEF7BF003
:020000040030CA
:0E000000FF38E2E2FFCEBBFFFFFFFFFFFFFF76
:0200000400F00A
:0400000000000000FC
:00000001FF
